:100000000C9437010C9454010C9454010C94540139
:100010000C9454010C9454010C9454010C9454010C
:100020000C9454010C9454010C9454010C945401FC
:100030000C94C3120C9454010C9454010C9454016C
:100040000C9454010C94B3050C94F4180C94D8112E
:100050000C9462120C9454010C9454010C945401AD
:100060000C9454010C9454010C9454010C945401BC
:100070004570692D4F5344205665722E302E392E0F
:10008000312E380000416B7475656C6C65732053BC
:10009000657474696E67000053657474696E6720D7
:1000A000200000486F6568656E73656E736F72201F
:1000B00000004853206D697420536368616C746557
:1000C0007220000048656164696E6720486F6C6447
:1000D0002000004B6F6D706173732000004B6F6DDB
:1000E0007061737320666978200000475053204187
:1000F0006B74697620000041636873656E6B6F7086
:1001000070656C756E67200000447265687261747A
:100110006520626567722E2000004665686C657216
:100120002046433C2D3E4F5344200000556E7465DD
:10013000727370616E6E756E672000004B65696E3C
:10014000652053657474696E672D416E7A656967C1
:1001500065000050432F425420616B7469760000A3
:1001600055656265726E65686D65204C65747A745C
:1001700065732053657474696E6700004B65696E22
:1001800065204465766976652D416E7A6569676597
:10019000000050432F425420616B74697600005573
:1001A000656265726E65686D65204C65747A74650C
:1001B000732044657669636500004F4E00002D2D65
:1001C0002D000044657669636520756E6420566570
:1001D0007273696F6E736162667261676500004475
:1001E000656369766520202020203D200000465769
:1001F0002D56657273696F6E203D200000464300E6
:10020000004E43000046432D6F6C642046570000AB
:100210004550492D4D656E750050616C0050432F5F
:100220004254004B656E6E756E670052432D4265F9
:100230007472696562004550492D5374726F6D0088
:1002400045786974004F4E002D2D0076767D7676C8
:100250007A76767E76767776767B76767876767C24
:1002600076767976767D76767A76767E7600112445
:100270001FBECFEFD4E0DEBFCDBF11E0A0E0B1E004
:10028000ECEFF3E302C005900D92AC38B107D9F75B
:1002900013E0ACE8B1E001C01D92AF3AB107E1F75D
:1002A0000E9464010C94FC190C94000086E981BB47
:1002B0008FE084BBAC9AAD9A8EE28ABB80EB87BBA1
:1002C000C69AD99ADD9A08951092D4011092D0015D
:1002D0001092D501E199FECF80E090E09FBB8EBBEC
:1002E000E09A8DB380939301E199FECF81E090E095
:1002F0009FBB8EBBE09A8DB380930001E199FECF46
:1003000082E090E09FBB8EBBE09A8DB38093940116
:10031000E199FECF87E190E09FBB8EBBE09A8DB361
:100320008093A101E199FECF88E190E09FBB8EBB55
:10033000E09A8DB38093BA01E199FECF8AE190E013
:100340009FBB8EBBE09A8DB380930901E199FECFEC
:1003500089E190E09FBB8EBBE09A8DB38093B6019C
:10036000E199FECF8BE190E09FBB8EBBE09A8DB30D
:100370008093950120910001213079F49EE09093C3
:10038000030187E08093040186E8809305012093B0
:100390000601909307018CE00EC09CE0909303014E
:1003A00085E0809304018AE48093050110920601A0
:1003B000909307018AE0809308010E941D170E9414
:1003C00056010E94AC0580919301813019F40E947E
:1003D000B31002C00E94A3107894A89A0E94E2046D
:1003E0000E9414060E94070A80919501882311F04B
:1003F0000E94470A8091BF01882311F00E94B41324
:100400000E94470A80919501813011F40E9444199D
:100410000E9484118091B201813021F41092B201C6
:100420000E94B4178091D901813021F41092D90132
:100430000E94DD0D80918E018130E9F410928E01D1
:100440008091D401882389F48091B601843069F4C5
:1004500080919301882349F480919601813029F499
:1004600080E363E64AE00E9432110E94B6120E94C5
:10047000BB120E94601480919501813031F480910B
:10048000DA01813011F40E944F198091910181307D
:10049000E1F48091D4018823C1F4AA9A0E94040F48
:1004A0000E9467090E947C088091BD01882321F089
:1004B0000E942F130E94C50A8091BE01882311F06B
:1004C0000E9465170E949C0AAA9880918C01813035
:1004D00069F58091D401882349F510928C018091AF
:1004E000A101882321F080910201833014F00E9441
:1004F000760A80919E0190919F01019690939F01B1
:1005000080939E010197CB9769F480919C01909113
:100510009D01019690939D0180939C0110929F01F3
:1005200010929E010E94550C0E949F0D80918D019A
:10053000813009F06FCF8091D401882309F06ACF10
:1005400010928D0180919501813039F48091DA010A
:10055000882319F481E00E944F190E94100A8091AB
:10056000BF01882309F456CF0E94E5130E9491131E
:1005700051CF782FD99827E030E041E050E0DB9868
:100580000000000000000000CA01022E02C0880F17
:10059000991F0A94E2F7872311F0DA9A01C0DA98DA
:1005A0000000000000000000DB9A000000000000D6
:1005B0000000215030408FEF2F3F380701F727E030
:1005C00030E041E050E0DB98000000000000000057
:1005D000CA01022E02C0880F991F0A94E2F78623EF
:1005E00011F0DA9A01C0DA98000000000000000063
:1005F000DB9A0000000000000000215030408FEF27
:100600002F3F380701F7DB98DA98D99A089584E0EC
:1006100064E00E94B90280E06CE40E94B90210928A
:100620008E0180918E018823E1F38CE66AE00E94BE
:10063000B90285E060E00E94B90208951F9380919D
:10064000B601823051F40E94C31010928C01809147
:100650008C018823E1F310928C0182E661E74FEF71
:100660000E94321110928C0110E00DC08091910116
:10067000813011F40E94040F80918C01813019F4B3
:1006800010928C0111E08091BC01882311F4112398
:1006900069F38091B601823011F40E940A1111238E
:1006A00009F0D9C080919E038093090180918E0347
:1006B0008093BA012091BA01E199FECF88E190E0E0
:1006C0009FBB8EBB2DBB0FB6F894E29AE19A0FBE8A
:1006D00020910901E199FECF8AE190E09FBB8EBB9A
:1006E0002DBB0FB6F894E29AE19A0FBE82E061E06A
:1006F00045E850E00E943F0E82E062E048E950E0A9
:100700000E943F0E82E064E043EA50E00E943F0E08
:1007100082E065E042EB50E00E943F0E82E066E03E
:1007200044EC50E00E943F0E82E067E043ED50E071
:100730000E943F0E82E068E04DED50E00E943F0EC7
:1007400082E069E04BEE50E00E943F0E82E06AE0FA
:1007500047EF50E00E943F0E82E06BE04CE251E038
:100760000E943F0E4091B8015091B90184E162E0CE
:100770000E94B20D8091BA0180FF05C084E164E05F
:100780004AEB51E004C084E164E04EEB51E00E948A
:100790003F0E8091BA0181FF05C084E165E04AEB1C
:1007A00051E004C084E165E04EEB51E00E943F0E51
:1007B0008091BA0182FF05C084E166E04AEB51E016
:1007C00004C084E166E04EEB51E00E943F0E809150
:1007D000BA0183FF05C084E167E04AEB51E004C041
:1007E00084E167E04EEB51E00E943F0E8091BA0138
:1007F00084FF05C084E168E04AEB51E004C084E175
:1008000068E04EEB51E00E943F0E8091BA0185FFF7
:1008100005C084E169E04AEB51E004C084E169E08D
:100820004EEB51E00E943F0E8091BA0186FF05C059
:1008300084E16AE04AEB51E004C084E16AE04EEBF7
:1008400051E00E943F0E4091090184E16BE050E0CD
:100850000E94B20D20C082E062E045E850E00E94B4
:100860003F0E82E065E04AE151E00E943F0EE199CF
:10087000FECF88E190E09FBB8EBBE09A8DB3809362
:100880008E03E199FECF8AE190E09FBB8EBBE09A98
:100890008DB38093090190918E03892F817080938D
:1008A000BD01892F88708093BE01892F807280934B
:1008B000BF0194709093C0011F9108951F93809180
:1008C0008C018823E1F310928C0183E666E740E017
:1008D0000E94321110E00DC080919101813011F41D
:1008E0000E94E70E80918C01813019F410928C01E6
:1008F00011E08091B701882311F4112369F31123CA
:1009000009F054C082E062E043EC51E00E943F0EE7
:1009100082E064E04FED51E00E943F0E82E066E02D
:100920004EEE51E00E943F0E8091B601813031F4CD
:100930008EE064E04DEF51E00E943F0E8091B601E1
:10094000823031F48EE064E041E052E00E943F0EDC
:100950008091B601843031F48EE064E045E052E0ED
:100960000E943F0E409148038EE066E050E00E94F6
:10097000B20D4091490380E166E050E00E94B20D63
:1009800040914A0383E166E050E00E94B20D20915D
:10099000B601E199FECF89E190E09FBB8EBB2DBBF4
:1009A0000FB6F894E29AE19A0FBE0AC0E199FECF21
:1009B00089E190E09FBB8EBBE09A8DB38093B60136
:1009C0001F9108950E94070383E66FE644E60E94A4
:1009D000321110928C0180918C018823E1F387E021
:1009E00062E040E750E00E943F0E0E941506109220
:1009F0008C0180918C018823E1F310928C0180910D
:100A00008C018823E1F310928C0180918C01882362
:100A1000E1F310928C0184E064E00E94B90280E06E
:100A20006CE40E94B90280919301882319F40E941A
:100A30005E041CC082E062E04CE751E00E943F0E81
:100A400082E064E042E951E00E943F0E82E066E00D
:100A50004FE951E00E943F0EE199FECF89E190E01D
:100A60009FBB8EBBE09A8DB38093B60180918C01C1
:100A70008823E1F310928C0180918C018823E1F3AB
:100A800010928C0184E064E00E94B90280E06CE482
:100A90000E94B90280919301882319F40E941E03D9
:100AA00026C082E062E04CE351E00E943F0E82E00B
:100AB00064E043E551E00E943F0E82E066E040E6DC
:100AC00051E00E943F0EE199FECF88E190E09FBB8C
:100AD0008EBBE09A8DB38093BA01E199FECF8AE193
:100AE00090E09FBB8EBBE09A8DB38093090180910B
:100AF000B601823029F483E66FE64AE00E943211A3
:100B00008091B601813029F482E664E64AE00E94D1
:100B1000321180918C018823E1F310928C01809135
:100B20008C018823E1F310928C0180918C01882341
:100B3000E1F310928C0180918C018823E1F31092F3
:100B40008C0180918C018823E1F310928C0184E068
:100B500064E00E94B902089582E083BF82E48EBD02
:100B60008AE089BF08951F920F920FB60F92112449
:100B70008F939F93809190018F5F809390018091DC
:100B80009001883449F591E090938F011092900183
:100B90008091A5038F5F8093A5038091A503843680
:100BA00031F41092A50390938C0190938D01809164
:100BB000A503823319F481E080938D018091A40311
:100BC0008F5F8093A4038091A4038A3029F410924C
:100BD000A40381E080938E019F918F910F900FBEAF
:100BE0000F901F901895982F80538A3010F020E0B6
:100BF00005C0903311F42AE001C0282F892F8154B9
:100C00008A3110F4292F2653892F81568A3110F406
:100C1000292F2C539D3211F429E403C09E3209F48C
:100C200021E4822F08950895089585E060E00E94F0
:100C3000B90286E063E80E94B90287E060E90E9499
:100C4000B90285E060E00E94B90286E064E80E9493
:100C5000B90287E061E90E94B90285E060E00E9484
:100C6000B90286E065E80E94B90287E062E90E9465
:100C7000B90285E060E00E94B90286E066E80E9461
:100C8000B90287E063E90E94B90285E060E00E9452
:100C9000B90286E067E80E94B90287E064E90E9431
:100CA000B90285E060E00E94B90286E068E80E942F
:100CB000B90287E065E90E94B90285E060E00E9420
:100CC000B90286E069E80E94B90287E066E90E94FD
:100CD000B90285E060E00E94B90286E06AE80E94FD
:100CE000B90287E067E90E94B90285E060E00E94EE
:100CF000B90286E061EA0E94B90287E068E90E94D1
:100D0000B90285E060E00E94B90286E062EA0E94D2
:100D1000B90287E069E90E94B90285E060E00E94BB
:100D2000B90286E063EA0E94B90287E06AE90E949C
:100D3000B90285E060E00E94B90286E064EA0E94A0
:100D4000B90287E06BE90E94B90285E060E00E9489
:100D5000B90286E065EA0E94B90287E06CE90E9468
:100D6000B90285E060E00E94B90286E066EA0E946E
:100D7000B90287E06DE90E94B90285E060E00E9457
:100D8000B90286E067EA0E94B90287E06EE90E9434
:100D9000B90285E060E00E94B90286E068EA0E943C
:100DA000B90287E06FE90E94B90285E060E00E9425
:100DB000B90286E06FEB0E94B90287E060EA0E9408
:100DC000B90285E060E00E94B90286E060EC0E9412
:100DD000B90287E061EA0E94B90285E060E00E9402
:100DE000B90286E061EC0E94B90287E062EA0E94E3
:100DF000B90285E060E00E94B90286E062EC0E94E0
:100E0000B90287E063EA0E94B90285E060E00E94CF
:100E1000B90286E063EC0E94B90287E064EA0E94AE
:100E2000B90285E060E00E94B90286E064EC0E94AD
:100E3000B90287E065EA0E94B90285E060E00E949D
:100E4000B90286E065EC0E94B90287E066EA0E947A
:100E5000B90285E060E00E94B90286E066EC0E947B
:100E6000B90287E067EA0E94B90285E060E00E946B
:100E7000B90286E06DED0E94B90287E068EA0E943F
:100E8000B90285E060E00E94B90286E06EED0E9442
:100E9000B90287E069EA0E94B90285E060E00E9439
:100EA000B90286E06FED0E94B90287E06AEA0E940B
:100EB000B90285E060E00E94B90286E060EE0E941F
:100EC000B90287E06BEA0E94B90285E060E00E9407
:100ED000B90286E061EE0E94B90287E06CEA0E94E6
:100EE000B90285E060E00E94B90286E062EE0E94ED
:100EF000B90287E06DEA0E94B90285E060E00E94D5
:100F0000B90286E063EE0E94B90287E06EEA0E94B1
:100F1000B90285E060E00E94B90286E064EE0E94BA
:100F2000B90287E06FEA0E94B90285E060E00E94A2
:100F3000B90286E06BEF0E94B90287E060EB0E9485
:100F4000B90285E060E00E94B90286E06CEF0E9481
:100F5000B90287E061EB0E94B90285E060E00E947F
:100F6000B90286E06DEF0E94B90287E062EB0E9451
:100F7000B90285E060E00E94B90286E06EEF0E944F
:100F8000B90287E063EB0E94B90285E060E00E944D
:100F9000B90286E06FEF0E94B90287E064EB0E941D
:100FA000B90285E061E00E94B90286E060E00E943B
:100FB000B90287E065EB0E94B90285E061E00E941A
:100FC000B90286E061E00E94B90287E066EB0E9408
:100FD000B9020895BF92CF92DF92EF92FF920F93E2
:100FE0001F93CF93DF937C01B62E8C0145E0C42E76
:100FF000D12CC80ED91E862F90E0EC01CC0FDD1F3E
:10100000C80FD91FCA5EDE4F0EC085E0612F0E9457
:10101000B90286E0602F0E94B90287E068810E94D1
:10102000B9020F5F1F4F0C151D0578F38701065F8E
:101030001F4F8FE090E0E80EF91E8B2D90E0EC0141
:10104000CC0FDD1FC80FD91FCA5EDE4F0EC085E072
:10105000612F0E94B90286E0602F0E94B90287E0EA
:1010600068810E94B9020F5F1F4F0E151F0578F3AC
:10107000DF91CF911F910F91FF90EF90DF90CF9074
:10108000BF900895EF92FF920F931F93CF93DF933A
:101090008C01EC0155E0E52EF12CE80EF91E0DC097
:1010A00085E06D2F0E94B90286E06C2F0E94B90284
:1010B00087E060E00E94B9022196CE15DF0580F33B
:1010C000E8012A96015F1F4F0DC085E06D2F0E9439
:1010D000B90286E06C2F0E94B90287E060E00E94AE
:1010E000B9022196C017D10780F3DF91CF911F91EC
:1010F0000F91FF90EF9008951F93CF93DF93C091CE
:101100004902D0914A02D7FD12C0CE016AE070E0D8
:101110000E94E919182F16952091040130E0CE01A4
:101120006AE070E00E94E919261B310918C0EE2719
:10113000FF27EC1BFD0BCF016AE070E00E94E9196C
:10114000182F16951C5F2091040130E02F5F3F4F50
:10115000CF016AE070E00E94E919260F311DE90114
:1011600075E0CC0FDD1F7A95E1F7220F331FC21B0C
:10117000D30B27968091120190911301C817D907BC
:1011800039F080911201909113010E94420804C02D
:101190008091C301811721F0CE01612F0E94EA07DF
:1011A0001093C301D0931301C0931201DF91CF912B
:1011B0001F910895CF92DF92EF92FF920F931F93AA
:1011C000CF93DF938C01E62E85E0612F0E94B90258
:1011D00086E0602F0E94B902CE2CDD2484E391E0EA
:1011E000C80ED91E87E0F60160810E94B902EEE1C7
:1011F000EE2EF12CE00EF11E85E06F2D0E94B9025B
:1012000086E06E2D0E94B90287E0F60160810E949F
:10121000B902E801CC54DF4F025F1E4F85E06D2F0D
:101220000E94B90286E06C2F0E94B90287E0F601A5
:1012300060810E94B9026E96C017D10779F7DF91DD
:10124000CF911F910F91FF90EF90DF90CF90089575
:10125000EF92FF920F931F93CF93DF937C0185E072
:101260006F2D0E94B90286E06E2D0E94B90287E0C0
:1012700060E00E94B9028701025E1F4F85E0612F86
:101280000E94B90286E0602F0E94B90287E060E008
:101290000E94B902E701CC54DF4F8701025F1E4F65
:1012A00085E06D2F0E94B90286E06C2F0E94B90282
:1012B00087E060E00E94B9026E96C017D10781F7FF
:1012C000DF91CF911F910F91FF90EF9008951F93A1
:1012D000CF93DF93E0914702F0914802F7FD14C0ED
:1012E000CF016AE070E00E94E919182F16951C5F83
:1012F00080910501C82FD0E0CF016AE070E00E9424
:10130000E919C61BD10917C0222733272E1B3F0B13
:10131000C9016AE070E00E94E919182F16958091C2
:101320000501C82FD0E02196C9016AE070E00E9453
:10133000E919C60FD11D8091140190911501C817AC
:10134000D90739F080911401909115010E94280964
:1013500004C08091C401811721F0CE01612F0E9449
:10136000DA081093C401D0931501C0931401DF91E2
:10137000CF911F91089585E060E00E94B90286E058
:101380006FEC0E94B90287E06CE80E94B90285E028
:1013900061E00E94B90286E06BE00E94B90287E03A
:1013A0006DE80E94B9020895EF92FF920F931F9388
:1013B000CF93DF937A019EE1699FB0011124680FFA
:1013C000711D8B01020F111D1092A603EB0115C0B8
:1013D00085E06D2F0E94B90286E06C2F0E94B90251
:1013E0008091A603F701E80FF11D60818F5F809364
:1013F000A60387E00E94B9022196C017D10740F3E7
:10140000DF91CF911F910F91FF90EF900895609120
:10141000030181E04DE051E025E00E94D4090895E8
:10142000DF93CF9300D000D0CDB7DEB7F8943091E2
:101430004F027894832F6AE00E94C919282F0E94D6
:10144000C919482F822F0E94C919292F832F0E9462
:10145000C919992319F48AE08C8301C09C83222343
:1014600019F48AE08A8301C02A83498385E48B8347
:1014700083E061E0AE014F5F5F4F24E00E94D4093A
:101480000F900F900F900F90CF91DF910895DF9301
:10149000CF9300D000D0CDB7DEB780E289839BE048
:1014A0009A8381E38B839C8381E061E0AE014F5F8F
:1014B0005F4F21E00E94D40980919501813079F439
:1014C00062E0AE014E5F5F4F21E00E94D40981E0EF
:1014D00063E0AE014D5F5F4F22E00E94D4090F90A0
:1014E0000F900F900F90CF91DF910895DF93CF93DE
:1014F00000D000D00F92CDB7DEB7DE011196E1E447
:10150000F1E085E001900D928150E1F760910401D6
:101510008CE0AE014F5F5F4F25E00E94D4090F9031
:101520000F900F900F900F90CF91DF91089580E072
:101530006CE40E94B902089580911C0390911D03F0
:10154000843B910554F080919E0390E020911A0312
:1015500030911B038217930744F08091C5018823C3
:1015600071F481E08093C50108958091C50118163A
:1015700024F480E06CE40E94B9021092C501089541
:1015800080E062E40E94B90208958F929F92AF9228
:10159000BF92CF92DF92EF92FF920F931F93DF9350
:1015A000CF93CDB7DEB72F970FB6F894DEBF0FBE3F
:1015B000CDBFFE013B9685E0DF011D928A95E9F7DC
:1015C00080914B0290914C026EE170E00E94E9190B
:1015D000CB01019797FF02C080E090E08E010F5F82
:1015E0001F4FB8014AE050E00E949819F80101909D
:1015F0000020E9F73197FE2EF01A80E0CF2CDD2491
:10160000C7FCD094F6E08F2E912C8C0E9D1E5801B5
:101610000BC0F501E00FF11F80810E94F305080D5A
:10162000191DF80180838E2D082F10E0E82EE39419
:101630000C151D0574F38093A60385E169E0AE01E6
:10164000455F5F4F25E00E94D40989E18F1969E069
:10165000A4012F2D0E94D4092F960FB6F894DEBF57
:101660000FBECDBFCF91DF911F910F91FF90EF90F3
:10167000DF90CF90BF90AF909F908F9008958F9202
:101680009F92AF92BF92CF92DF92EF92FF920F9311
:101690001F93DF93CF93CDB7DEB72E970FB6F89495
:1016A000DEBF0FBECDBF19821A821B821C828091C1
:1016B000AA019091AB018E010B5F1F4FB8014AE068
:1016C00050E00E949819F80101900020E9F7319745
:1016D000FE2EF01A80E0CF2CDD24C7FCD094AAE0C7
:1016E0008A2E912C8C0E9D1E58010BC0F501E00F27
:1016F000F11F80810E94F305080D191DF8018083F8
:101700008E2D082F10E0E82EE3940C151D0574F3C0
:101710008093A60385E166E0AE014F5F5F4F24E052
:101720000E94D40989E18F1966E0A4012F2D0E943F
:10173000D4098091AA019091AB011816190664F49E
:1017400085E060E00E94B90286E062EC0E94B90286
:1017500087E06CE80E94B9028091AA019091AB01E8
:1017600097FF0CC085E060E00E94B90286E062EC61
:101770000E94B90287E06DE80E94B9028091AA0137
:101780009091AB01892B61F485E060E00E94B90281
:1017900086E062EC0E94B90287E060E00E94B90234
:1017A0002E960FB6F894DEBF0FBECDBFCF91DF915E
:1017B0001F910F91FF90EF90DF90CF90BF90AF906F
:1017C0009F908F9008958F929F92AF92BF92CF92E9
:1017D000DF92EF92FF920F931F93DF93CF93CDB7DA
:1017E000DEB72B970FB6F894DEBF0FBECDBFDE017C
:1017F0001196EEE3F1E083E001900D928150E1F764
:101800008E010C5F1F4F8091180390911903B8014E
:101810004AE050E00E949819F80101900020E9F791
:101820003197FE2EF01A80E0CF2CDD24C7FCD09437
:10183000B8E08B2E912C8C0E9D1E58010BC0F5012B
:10184000E00FF11F80810E94F305080D191DF801BA
:1018500080838E2D082F10E0E82EE3940C151D05D3
:1018600074F38093A6038DE06EE0AE014F5F5F4F8F
:1018700023E00E94D40980E18F196EE0A4012F2D8E
:101880000E94D4092B960FB6F894DEBF0FBECDBFD1
:10189000CF91DF911F910F91FF90EF90DF90CF904C
:1018A000BF90AF909F908F9008958F929F92AF922C
:1018B000BF92DF92EF92FF920F931F93DF93CF932C
:1018C000CDB7DEB728970FB6F894DEBF0FBECDBFF9
:1018D00019828AE08A8380919C0190919D018E01FA
:1018E0000D5F1F4FB8014AE050E00E949819F801BF
:1018F00001900020E9F73197E01B80E0EE2EFF24F5
:10190000E7FCF094480106E0A02EB12CAC0EBD1E01
:101910000BC0F401E00FF11F80810E94F3050A0D56
:101920001B1DF80180838D2D082F10E0D82ED39435
:101930000E151F0574F38093A60380919C0190916E
:101940009D018E010A5F1F4F0A977CF4609103018D
:1019500081E0AE014F5F5F4F21E00E94D4096091AA
:10196000030182E0A80121E005C06091030181E04C
:10197000A80122E00E94D40980919E0190919F01CC
:101980008E010D5F1F4FB8014AE050E00E94981988
:10199000F80101900020E9F73197E01B80E0EE2E7E
:1019A000FF24E7FCF094480116E0A12EB12CAC0E08
:1019B000BD1E0BC0F401E00FF11F80810E94F305F2
:1019C0000A0D1B1DF80180838D2D082F10E0D82EE5
:1019D000D3940E151F0574F38093A60380919E0186
:1019E00090919F018E010A5F1F4F0A977CF46091CE
:1019F000030184E0AE014E5F5F4F21E00E94D409F5
:101A00006091030185E0A80121E005C06091030118
:101A100084E0A80122E00E94D40928960FB6F89429
:101A2000DEBF0FBECDBFCF91DF911F910F91FF9011
:101A3000EF90DF90BF90AF909F908F9008950F939D
:101A40001F93DF93CF93CDB7DEB72A970FB6F894E5
:101A5000DEBF0FBECDBF8E010F5F1F4FB8014AE042
:101A600050E00E949819F80101900020E9F73197A1
:101A7000E01B20E0FF27E7FDF095322F3F5F822F2C
:101A800090E08E179F0714F4232FF7CF2093A6031F
:101A90002A960FB6F894DEBF0FBECDBFCF91DF916F
:101AA0001F910F910895AF92BF92CF92DF92EF9264
:101AB000FF920F931F93DF93CF93CDB7DEB76E974F
:101AC0000FB6F894DEBF0FBECDBFB82EA62ED42E13
:101AD000A42FB52FFD0101900020E9F73197CE2EFC
:101AE000C41A7E010894E11CF11C242F352FC90172
:101AF0008C0108C0F80181918F010E94F305F70164
:101B000081937F01802F8D198C15A0F38B2D6A2D69
:101B1000AE014F5F5F4F2C2D0E94D4096E960FB619
:101B2000F894DEBF0FBECDBFCF91DF911F910F9113
:101B3000FF90EF90DF90CF90BF90AF90089580918D
:101B40009401813071F4609106012091DB013091A4
:101B5000DC01369527958EE0821B4DED51E00E9409
:101B6000530D0895EF92FF920F931F93DF93CF933E
:101B7000CDB7DEB764970FB6F894DEBF0FBECDBF0A
:101B8000F82EE62ECA018E010F5F1F4FB8014AE002
:101B900050E00E9498198F2D6E2DA8010E94530DC0
:101BA00064960FB6F894DEBF0FBECDBFCF91DF9124
:101BB0001F910F91FF90EF900895EF92FF920F9376
:101BC0001F93DF93CF93CDB7DEB72A970FB6F89464
:101BD000DEBF0FBECDBF20915703822F6AE00E9467
:101BE000C919382F822F0E94C91985E48F838091EB
:101BF0005803882309F48AE08887992319F48AE036
:101C00008E8301C09E833D8319821A821B821C82AF
:101C10008E010B5F1F4F83E062E0A80124E00E9469
:101C2000D40980915B0390915C03B8014AE050E0D5
:101C30000E949819F80101900020E9F77F010894AB
:101C4000E108F108E01AF10A83E063E0AE014F5FBA
:101C50005F4F24E00E94D40987E08E1963E0A80159
:101C60000E94530D2A960FB6F894DEBF0FBECDBF6B
:101C7000CF91DF911F910F91FF90EF900895BF9248
:101C8000CF92DF92EF92FF920F931F93DF93CF9348
:101C9000CDB7DEB764970FB6F894DEBF0FBECDBFE9
:101CA000C82EB62EFA017E010894E11CF11C04C076
:101CB000AE0DBF1D9C9331968E2F841B9491A82F3F
:101CC000B0E09923A9F7AE0DBF1D1C92F70101905A
:101CD0000020E9F73197DE2EDE18870107C0F801F2
:101CE00080810E94F305F80181938F01802F8E1966
:101CF0008D15A8F38C2D6B2DAE014F5F5F4F2D2DF1
:101D00000E94D40964960FB6F894DEBF0FBECDBF13
:101D1000CF91DF911F910F91FF90EF90DF90CF90C7
:101D2000BF9008951F93CF93DF93EC01A3E0B0E041
:101D300047C0FD01E059FD4F8081FD01EF58FD4F87
:101D40002081422F50E04D535040FD01EE58FD4F91
:101D50007081FD01ED58FD4F10819A01F4E0359539
:101D60002795FA95E1F790E0CD97880F991F880F96
:101D7000991F282B392B2883613029F1E72FF0E0B8
:101D8000FD9734E0440F551F3A95E1F75070CF01AD
:101D90009595879595958795482B592B4983623062
:101DA00091F01496635086E0EE0FFF1F8A95E1F7DD
:101DB000F070812F90E0CD97E82BF92BEA832396E2
:101DC000662309F0B6CFDF91CF911F9108958091DE
:101DD00072028635B1F48091710281568093B6010A
:101DE0008091B601843018F084E08093B60188E4D5
:101DF00093E06AE043E02AE00E94920E81E0809343
:101E0000B7011092910108951F931091B6011230FD
:101E100009F482C0143009F4D3C0113009F08FC125
:101E200080917202813581F484E893E06BE143E0B4
:101E30002DE20E94920E8091840390E09093B9016C
:101E40008093B8011093BC0180917202843409F030
:101E500076C186E093E061E443E021E40E94920EC3
:101E600080911C0390911D03843B910554F4809153
:101E70009601813031F410929601F8940E94B310CB
:101E8000789480911C0390911D03843B91057CF014
:101E900080919601882359F481E080939601F8940B
:101EA00080919301882311F40E94A310789480916B
:101EB00008039091090366E170E00E94E9196E5FE2
:101EC0007F4F70934A026093490280910A03909178
:101ED0000B0366E170E00E94E9196A5F7F4F70931F
:101EE00048026093470280911203909113039093EC
:101EF0004C0280934B0280911A0380934F02809191
:101F00002E0290912F0290934E0280934D02809169
:101F100018038093510213C1809172028F34A9F08B
:101F2000813509F00CC184E893E06CE143E02DE2D7
:101F30000E94920E8091840390E09093B901809367
:101F4000B80181E08093BC01FAC081EF91E060E5C7
:101F500043E02DE20E94920E80913902992787FD7D
:101F60009095029690934A028093490280913A029A
:101F7000992787FD90950696909348028093470293
:101F800080912C0290912D0290934C0280934B02F1
:101F90008091320280934F0280912E0290912F0205
:101FA00090934E0280934D028091370280935102AC
:101FB00080912B028093520281E08093BB01BFC0CD
:101FC00080917202843409F056C086E093E061E4A7
:101FD00043E021E40E94920E80911C0390911D0326
:101FE000843B910554F480919601813031F4109234
:101FF0009601F8940E94B310789480911C039091FC
:102000001D03843B91057CF080919601882359F44F
:1020100081E080939601F89480919301882311F4D4
:102020000E94A3107894809108039091090366E1BF
:1020300070E00E94E9196E5F7F4F70934A026093CF
:10204000490280910A0390910B0366E170E00E94BF
:10205000E9196A5F7F4F709348026093470280914D
:1020600012039091130390934C0280934B02809142
:10207000180380935102809172028C3481F481E0C4
:1020800090E09093B9018093B80181E08093BC0106
:1020900086E893E069E143E02DE20E94920E809190
:1020A00072028D3481F482E090E09093B9018093C4
:1020B000B80181E08093BC0186E893E069E143E0E8
:1020C0002DE20E94920E809172028E3481F483E0A0
:1020D00090E09093B9018093B80181E08093BC01B6
:1020E00086E893E069E143E02DE20E94920E809140
:1020F00072028F3481F484E090E09093B901809370
:10210000B80181E08093BC0186E893E069E143E097
:102110002DE20E94920E80917202803581F485E05A
:1021200090E09093B9018093B80181E08093BC0165
:1021300086E893E069E143E02DE20E94920E10925E
:1021400091011F91089582E289B910BC80B91CBE2B
:10215000909A28E92AB996E890BD82EC8BB921B90A
:102160009CBF82B9089582E289B910BC80B91CBEB7
:1021700088E98AB926E820BD92EC9BB980E981B94B
:102180002CBF92B90895DF93CF93CDB7DEB72C97CC
:102190000FB6F894DEBF0FBECDBF83E2898383E61E
:1021A0008A8385E78B838DE38C838D838E838F83F6
:1021B000DE011196FD0120E030E0AE01485F5F4F87
:1021C0008191280F311DE417F507D1F7C9019F70E0
:1021D00046E0959587954A95E1F7835C88872F734C
:1021E0003070822F835C89878DE08A879E01255F0E
:1021F0003F4F8C91159BFECF83B91196A217B30761
:10220000C1F72C960FB6F894DEBF0FBECDBFCF91AD
:10221000DF910895DF93CF93CDB7DEB72C970FB63C
:10222000F894DEBF0FBECDBF8BE189838A8385E53D
:102230008B838AEA8C831D82FE0131969E012A5F80
:102240003F4F8081159BFECF83B93196E217F3078C
:10225000C1F72C960FB6F894DEBF0FBECDBFCF915D
:10226000DF910895DF93CF93CDB7DEB72A970FB6EE
:10227000F894DEBF0FBECDBF93E299838A836B8350
:10228000842F86958695835C8C8350E043705070D4
:1022900064E0440F551F6A95E1F7435C4D838DE37D
:1022A0008E838F83DE011196FD0120E030E0AE01C8
:1022B000485F5F4F8191280F311DE417F507D1F773
:1022C000C9019F7056E0959587955A95E1F7835C13
:1022D00088872F733070822F835C89878DE08A878F
:1022E0009E01255F3F4F8C91159BFECF83B91196C0
:1022F000A217B307C1F72A960FB6F894DEBF0FBE38
:10230000CDBFCF91DF9108955D9BFECF8DE68CB957
:102310005D9BFECF8FE68CB95D9BFECF89E68CB9C5
:102320005D9BFECF8EE68CB95D9BFECF8DE08CB9B8
:102330005D9BFECF8EE38CB90895982F9F70829598
:102340008F708A3010F4805D01C0895C5D9BFECF88
:102350008CB99A3018F4892F805D02C0892F895C6E
:102360005D9BFECF8CB908958A3010F4805D01C06A
:10237000895C5D9BFECF8CB90895159BFECF83B918
:1023800008955D9BFECF8CB90895662359F020E037
:10239000FC01E20FF11DE0815D9BFECFECB92F5FE8
:1023A0006217B0F708955D9BFECF8EE38CB9089558
:1023B0001F920F920FB60F9211242F933F938F937A
:1023C0009F93AF93BF93EF93FF932CB12093A703F9
:1023D00085B398E0892785BB5D9BFECF2CB92D3056
:1023E00059F080918303E82FF0E0E35AFC4F2083FB
:1023F0008F5F8093830359C0E0918303F0E0E35A39
:10240000FC4F20831092B3011092B4011092B501D9
:1024100030E020E090E03FC02130B9F0213018F0EA
:102420002230C1F524C0A32FB0E0A35ABC4F8C9139
:10243000803211F421E023C0E92FF0E08C91E558BF
:10244000FC4F80839093B30124C0A32FB0E0A35A24
:10245000BC4F8C91803211F422E011C0E92FF0E0E2
:102460008C91ED59FD4F80839093B40112C0A32F3E
:10247000B0E0A35ABC4F8C91803219F423E090E075
:1024800009C0E92FF0E08C91EC5AFD4F80839093C6
:10249000B5019F5F3F5F80918303831708F0BCCF36
:1024A00081E08093B20110928303FF91EF91BF917D
:1024B000AF919F918F913F912F910F900FBE0F90F1
:1024C0001F9018951F920F920FB60F9211248F93A1
:1024D0009F93EF93FF9393B19093A8039D3081F462
:1024E0008091C601813061F4AB981092C60180934F
:1024F0009101E0915303F0E0E059FD4F90832DC02E
:102500008091C601882319F0813039F514C09332C7
:1025100041F480919101882321F481E08093C601E8
:10252000AB9A1092530380915303E82FF0E0E059E7
:10253000FD4F90830CC0E0915303F0E0E059FD4F54
:10254000908380915303853930F4809153038F5FDA
:102550008093530302C01092C601FF91EF919F91A7
:102560008F910F900FBE0F901F90189585B392E03A
:10257000892785BB089590919901913019F485B30D
:10258000892785BB08951F920F920FB60F921124D1
:102590002F933F935F936F937F938F939F93AF930B
:1025A000BF938091C8019091C901892B81F484B5B2
:1025B00095B59093CF018093CE018EB58F7B8EBD64
:1025C00081E090E09093C9018093C8013AC084B53E
:1025D00095B59093CD018093CC012EB520642EBD8E
:1025E0002091CE013091CF011092C9011092C80103
:1025F000821B930B865698406CE271E00E94D519BD
:102600007093CB016093CA016730710534F086E0A6
:1026100090E09093CB018093CA012091CA01309140
:10262000CB0180910201992787FD909528173907E2
:1026300041F0263031052CF42093020181E0809393
:10264000A001BF91AF919F918F917F916F915F9109
:102650003F912F910F900FBE0F901F901895809172
:102660004B0290914C029093A3018093A201809120
:10267000A2019091A3012091A4013091A501821B98
:10268000930B9093A7018093A6018091A201909152
:10269000A3019093A5018093A4014091AE015091B4
:1026A000AF018091A6019091A701E3E0880F991FE7
:1026B000EA95E1F79A0173E0220F331F7A95E1F76B
:1026C000241B350B820F931F68E070E00E94E9190C
:1026D0007093AF016093AE012091B0013091B101D0
:1026E0004091AE015091AF01C90163E0880F991F7D
:1026F0006A95E1F7821B930B840F951F68E070E0E9
:102700000E94E9197093B1016093B0018091B0010A
:102710009091B1019093AB018093AA010E943F0B6D
:102720000895DF93CF930F92CDB7DEB78091270244
:102730009091280221E0823592071CF080EC898379
:1027400006C06DE270E00E94E919605469836091EF
:1027500004018EE0AE014F5F5F4F21E00E94D4097B
:102760000F90CF91DF9108958AE161E04EE451E04E
:1027700022E00E94D4090895DF93CF9300D00F92F6
:10278000CDB7DEB7DE011196E0E5F1E083E0019020
:102790000D928150E1F7609104016F5F8EE0AE0110
:1027A0004F5F5F4F23E00E94D409609104016F5F87
:1027B00040912502509126028EE00E94B20D0F90AA
:1027C0000F900F90CF91DF9108958F929F92BF92BB
:1027D000CF92DF92EF92FF920F931F93DF93CF93ED
:1027E000CDB7DEB72B970FB6F894DEBF0FBECDBFC7
:1027F000DE011196E3E5F1E083E001900D92815056
:10280000E1F7809152028E010C5F1F4F90E0B801FA
:102810004AE050E00E949819F80101900020E9F781
:102820003197BE2EB01AEE24FF24CB2CDD24C7FC3A
:10283000D09488E0882E912C8C0E9D1E0DC0F8013E
:10284000EE0DFF1D80810E94F305F401EE0DFF1DCA
:1028500080830894E11CF11CEC14FD0484F388E1EE
:1028600061E0AE014F5F5F4F23E00E94D4098BE12E
:102870008B1961E0A4012B2D0E94D4092B960FB671
:10288000F894DEBF0FBECDBFCF91DF911F910F91A6
:10289000FF90EF90DF90CF90BF909F908F90089522
:1028A00083E66FE644E60E943211F89428E088E15E
:1028B00090E00FB6F894A89581BD0FBE21BDFFCF63
:1028C0001F939D998AC18091D0018F5F8093D00121
:1028D00011E01093D2018091D001853009F081C1BF
:1028E0008091D401882309F08CC01093D4011092F8
:1028F000D50184E064E00E94B90283E061E04DED1F
:1029000051E00E94530D83E063E040E152E00E94F9
:102910003F0E84E068E00E94B90283E065E049E18F
:1029200052E00E943F0E80910001813029F484E141
:1029300065E045E452E004C084E165E048E452E02B
:102940000E943F0E84E060E00E94B90283E066E0EE
:102950004DE152E00E943F0E80919301813029F4B5
:1029600084E166E045E452E004C084E166E048E4C6
:1029700052E00E943F0E83E067E043E252E00E9493
:102980003F0E80919401813029F484E167E045E4B1
:1029900052E004C084E167E048E452E00E943F0E48
:1029A00083E068E04BE252E00E943F0E8091A1017B
:1029B000813029F484E168E045E452E004C084E118
:1029C00068E048E452E00E943F0E83E069E046E39D
:1029D00052E00E943F0E80919501813029F484E1FC
:1029E00069E045E452E004C084E169E048E452E073
:1029F0000E943F0E83E06BE040E452E00E943F0EF5
:102A0000EEC08091D501882349F584E068E00E94FA
:102A1000B90280910001882339F41093000184E108
:102A200065E045E452E006C01092000184E165E0F3
:102A300048E452E00E943F0E20910001E199FECF50
:102A400081E090E09FBB8EBB2DBB0FB6F894E29A5D
:102A5000E19A0FBE84E060E00E94B9021091D501B6
:102A6000113049F584E068E00E94B9028091930139
:102A7000882339F41093930184E166E045E452E041
:102A800006C01092930184E166E048E452E00E949F
:102A90003F0E20919301E199FECF80E090E09FBB33
:102AA0008EBB2DBB0FB6F894E29AE19A0FBE84E07C
:102AB00060E00E94B9028091D501823051F584E036
:102AC00068E00E94B90280919401882341F481E07A
:102AD0008093940184E167E045E452E006C01092DF
:102AE000940184E167E048E452E00E943F0E2091A7
:102AF0009401E199FECF82E090E09FBB8EBB2DBB9D
:102B00000FB6F894E29AE19A0FBE84E060E00E946A
:102B1000B9028091D501833051F584E068E00E94CC
:102B2000B9028091A101882341F481E08093A10141
:102B300084E168E045E452E006C01092A10184E11E
:102B400068E048E452E00E943F0E2091A101E19923
:102B5000FECF87E190E09FBB8EBB2DBB0FB6F894F4
:102B6000E29AE19A0FBE84E060E00E94B90280918F
:102B7000D501843049F568E00E94B9028091950141
:102B8000882341F481E08093950184E169E045E484
:102B900052E006C01092950184E169E048E452E0F9
:102BA0000E943F0E20919501E199FECF8BE190E0CC
:102BB0009FBB8EBB2DBB0FB6F894E29AE19A0FBE75
:102BC00084E060E00E94B9028091D501853049F42B
:102BD0001092D4010E94501404C01092D00110929F
:102BE000D2019C9913C19091D401913009F014C184
:102BF0009093D3018091D1018F5F8093D101209177
:102C0000D101253009F008C11092D1018091D50180
:102C1000823009F469C0833030F4882371F0813048
:102C200009F0FAC035C0843009F4AAC0843008F431
:102C300086C0853009F0F0C0C3C09093D50183E011
:102C400065E049E152E00E943F0E80910001813031
:102C500029F484E165E045E452E004C084E165E0E4
:102C600048E452E00E943F0E84E068E00E94B9020E
:102C700083E066E04DE152E00E943F0E80919301B7
:102C8000813019F484E166E0B3C084E166E0B5C048
:102C900082E08093D50183E066E04DE152E00E943E
:102CA0003F0E80919301813029F484E166E045E490
:102CB00052E004C084E166E048E452E00E943F0E26
:102CC00084E068E00E94B90283E067E043E252E0FA
:102CD0000E943F0E80919401813019F484E167E0F5
:102CE00087C084E167E089C083E08093D50167E015
:102CF00043E252E00E943F0E80919401813029F41A
:102D000084E167E045E452E004C084E167E048E420
:102D100052E00E943F0E84E068E00E94B90283E026
:102D200068E04BE252E00E943F0E8091A1018130A9
:102D300019F484E168E05CC084E168E05EC084E08E
:102D40008093D50183E068E04BE252E00E943F0EA1
:102D50008091A101813029F484E168E045E452E0EA
:102D600004C084E168E048E452E00E943F0E84E041
:102D700068E00E94B90283E069E046E352E03FC0A8
:102D80002093D50183E069E046E352E00E943F0EC4
:102D900080919501813029F484E169E045E452E0B5
:102DA00004C084E169E048E452E00E943F0E84E000
:102DB00068E00E94B90283E06BE040E452E01FC08B
:102DC0001092D50183E06BE040E452E00E943F0E98
:102DD00084E068E00E94B90283E065E049E152E0E6
:102DE0000E943F0E80910001813029F484E165E06A
:102DF00045E452E004C084E165E048E452E00E940A
:102E00003F0E84E060E00E94B90206C01092D1013A
:102E10008091D2018091D3011F910895813061F496
:102E2000E199FECF80E090E09FBB8EBB6DBB0FB6FB
:102E3000F894E29AE19A0FBE0895DF93CF93CDB74D
:102E4000DEB764970FB6F894DEBF0FBECDBF20E0AB
:102E5000DE011196E199FECFE22FF0E0CF018D5F08
:102E60009F4F9FBB8EBBE09A8DB3EA0FFB1F808301
:102E7000882311F02F5FEECFFD0101900020E9F7CC
:102E80009F01215030402A1B3B0B3093DC012093E3
:102E9000DB0190E0AE014F5F5F4F09C0FD01E352DF
:102EA000FE4FA40FB51F8C91808311829F5FA92FC5
:102EB000B0E0A217B30790F364960FB6F894DEBFA4
:102EC0000FBECDBFCF91DF910895DF93CF93CDB7E4
:102ED000DEB760970FB6F894DEBF0FBECDBF80910E
:102EE000510290E090936F0280936E0280916E0287
:102EF00090916F026FE070E00E94D519DE01159687
:102F0000AD016A1B9E01205F3F4FE62FEA0FF0E004
:102F1000E55BFD4FE491ED93A217B307B1F7609124
:102F2000070119821A821B821C8289E02BE00E9411
:102F3000D409609108018EE0AE014F5F5F4F24E03D
:102F40000E94D4096091080140916E0250916F0275
:102F50008FE00E94B20D60960FB6F894DEBF0FBEF0
:102F6000CDBFCF91DF910895DF93CF93CDB7DEB77B
:102F7000E2970FB6F894DEBF0FBECDBFDE01179605
:102F8000E6E5F1E087E001900D928150E1F7DE0186
:102F90001E96EDE5F1E089E001900D928150E1F798
:102FA000DE015796E6E6F1E08EE001900D92815049
:102FB000E1F7DE011196E4E7F1E086E001900D9281
:102FC0008150E1F7DE019596EAE7F1E08EE00190AD
:102FD0000D928150E1F750917B0360917C03409109
:102FE0007D0380917E0320E030E0803711F421E002
:102FF00030E080E090E04C3611F481E090E028234E
:10300000392380E0583609F481E090E0653609F410
:1030100091E0892390E028233923232B79F0CE01F6
:10302000079666E00E94C511CE010E9668E00E94E8
:10303000C511CE0147966DE00E94C51150917B03EA
:1030400060917C0340917D0380917E0320E030E01D
:10305000873711F421E030E080E090E04F3611F442
:1030600081E090E02823392380E0533709F481E0A0
:1030700090E0683609F491E0892390E02823392311
:10308000232B19F18091630290916402893481F4B9
:10309000943471F4CE01019665E00E94C5118DED66
:1030A00091E06091DB010E94C5118DE00E94C11189
:1030B0008091630290916402863739F4953629F441
:1030C000CE0185966CE00E94C51180917B03209112
:1030D0007C0340917D0390E0833709F491E080E028
:1030E000253609F481E09823892F90E020E030E034
:1030F000443711F421E030E082239323892B09F433
:1031000042C08091630290916402893409F03BC00F
:10311000943409F038C020E01AC0FD01EC5AFD4F8C
:10312000E081E199FECF822F90E08D5F9F4F9FBBA2
:103130008EBBEDBB0FB6F894E29AE19A0FBEFD018B
:10314000EC5AFD4F8081A352BE4F8C932F5F80912C
:10315000B501A22FB0E0281700F3E199FECFCD0111
:103160008D5F9F4F9FBB8EBB1DBA0FB6F894E29A3E
:10317000E19A0FBEE22FF0E0E352FE4F1082B093CF
:10318000DC01A093DB0150917B0360917C034091B3
:103190007D0380917E0320E030E0853611F421E04C
:1031A00030E080E090E0433711F481E090E02823A4
:1031B000392380E0523709F481E090E0653609F464
:1031C00091E0892390E028233923232B11F00E94DA
:1031D00050140E94D311E2960FB6F894DEBF0FBED2
:1031E000CDBFCF91DF9108951F920F920FB60F922E
:1031F00011242F933F938F939F93EF93FF9380918D
:10320000D701882381F08091D70190E00197E09168
:103210008A01F0918B01E80FF91F8FB1808381E063
:103220008093D80103C08FB18093AE032091D70162
:103230008091880130E0992787FD90958217930748
:103240005CF084E08093890181E08093D8018091D3
:10325000D7018093AD0308C0929A1092D60181E005
:103260008093D9011092DA018091D7018F5F80930A
:10327000D701FF91EF919F918F913F912F910F90E7
:103280000FBE0F901F90189582ED8DB90895813073
:1032900029F4613011F492980895929A0895982F24
:1032A0008091D6018823C9F4913009F492989093C3
:1032B000D60181E08093DA01913069F486E0809351
:1032C00088011092D7018AE0809389019093D801F8
:1032D0008AEA8093AD0380E008958091D80181301F
:1032E00071F4809189018150809389018F5F39F455
:1032F0008091AD038FB91092D80181E0089581E0EB
:103300000895CF93DF93C0E0D0E0E0918A01F0917F
:103310008B01EC0FFD1F80810E949D112196C7300B
:10332000D10599F78DE00E94C111DF91CF910895E9
:10333000FB019F01E8944230C4F04532B4F44A30B6
:1033400029F497FB1EF4909581959F4F642F772762
:103350000E94D519805D8A330CF0895D8193CB0181
:103360000097A1F716F45DE251931082C9010C9405
:10337000B919DC01FC01672F71917723E1F73297CE
:1033800004C07C916D9370836291AE17BF07C8F340
:103390000895991B79E004C0991F961708F0961BB1
:1033A000881F7A95C9F780950895AA1BBB1B51E128
:1033B00007C0AA1FBB1FA617B70710F0A61BB70BA5
:1033C000881F991F5A95A9F780959095BC01CD014A
:1033D000089597FB092E07260AD077FD04D0E5DF74
:1033E00006D000201AF4709561957F4F0895F6F786
:0C33F000909581959F4F0895F894FFCFB1
:1033FC000101030E0786010E0C5C00000A0000445C
:10340C00000023002300546466536365526200512C
:10341C0061005060005060005161005262005363C3
:10342C00655464666768696A6B6B6A6968670000F3
:10343C000053536353530603F10184030D0A0A1D11
:10344C0000000000000068656C70200D0073686F50
:10345C00772049440D0073686F7720766572736925
:10346C006F6E0D004944203D2000302E392E312E38
:0C347C00382E626574610D0009075603CC
:00000001FF
